:100000000C94A0000C9448010C946D010C94920186
:100010000C94BB000C94BB000C94BB000C94BB0074
:100020000C94BB000C94BB000C94BB000C94DB0E36
:100030000C94130F0C94BB000C94D6030C94BB00CF
:100040000C94BB000C94BB000C94BB000C94BB0044
:100050000C94BB000672652C0375223B59781EBABE
:10006000E07A633BF47C75FF4E7E3172117F0000B5
:10007000000005813504F483200001836246328349
:10008000200000816246307F0000000582778C4F9F
:1000900081432CE28217BF2483A48DD981E1D8A1AA
:1000A00080DB67820000000D416C6C20726967681C
:1000B00074732072657365727665642E006C756B5F
:1000C00061737A40776F6269742E636F6D2E706C06
:1000D0000D004D617465636B690D6C757465636BC0
:1000E00069406F702E706C0D00436F707972696794
:1000F00068742028632920323030350D4C756B61CF
:10010000737A20005245562E3A20312E3620004672
:100110004C4153483A200031323A32343A323300BB
:100120004465632020322032303035002C200057C7
:100130004F62697420534443313036452C2000000F
:1001400011241FBECFE5D4E0DEBFCDBF10E0A0E696
:10015000B0E0E0ECFBE202C005900D92AC37B107D5
:10016000D9F712E0ACE7B0E001C01D92A435B107A9
:10017000E1F70C9418020C9400001ABA8FEF87BBB9
:1001800084BB81BB08950895BB9A84B3836084BB0C
:10019000A298AA9A13BE83B7896683BF08959B016C
:1001A000AC01211531054105510549F080EA9FE078
:1001B0000197F1F72150304040405040F2CF089570
:1001C0000F931F93CF93DF93EC019A9927C0F89474
:1001D000A898A9981CBE83B38074082F112783B3F5
:1001E0009927807490700817190761F4A89582B355
:1001F00090E2892782BB6AEF70E080E090E00E9485
:10020000CF00EDCF68EE73E080E090E00E94CF0079
:10021000959A789480E293E00197F1F780917C00C1
:1002200090917D00C89F9001C99F300DD89F300DDF
:100230001124121613068CF01CBE80E293E0019785
:10024000F1F7A898A99880E293E00197F1F7A89AAE
:10025000A99A80E991E00197F1F71C161D061CF49C
:10026000A89AA99804C0D7FF02C0A898A99ACE015D
:10027000D7FF04C0882799278C1B9D0B8CBFD09378
:100280007D00C0937C00DF91CF911F910F91089565
:100290001F920F920FB60F9211248F939F93AF93DB
:1002A000BF938091420190914301A0914401B0918C
:1002B00045010196A11DB11D809342019093430118
:1002C000A0934401B0934501BF91AF919F918F914D
:1002D0000F900FBE0F901F9018951F920F920FB6A0
:1002E0000F9211248F939F93AF93BF9380914201FC
:1002F00090914301A0914401B09145010197A1095A
:10030000B1098093420190934301A0934401B093BB
:100310004501BF91AF919F918F910F900FBE0F90AC
:100320001F9018951F920F920FB60F9211242F93C2
:100330003F934F935F936F937F938F939F93AF936D
:10034000BF93EF93FF93A895809142019091430151
:10035000A0914401B09145018093E8009093E90099
:10036000A093EA00B093EB0078949F9904C081E0D9
:100370008093E30002C01092E3009E9B04C081E0E2
:100380008093DD0002C01092DD0084EE90E00E94B8
:10039000F605609100017091010180910201909138
:1003A00003010E947913DC01CB01BC01CD010E9445
:1003B0005213DC01CB010E94E00088B7806888BF3F
:1003C000FF91EF91BF91AF919F918F917F916F912D
:1003D0005F914F913F912F910F900FBE0F901F9003
:1003E00018950F931F938C01C801AA2797FDA0951C
:1003F000BA2FBC01CD010E946F1317FF06C020E089
:1004000030E040E857E40E94311220E030E04AE753
:1004100055E40E940714DC01CB01BC01CD010E9410
:100420005213DC01CB010197F1F71F910F91089551
:10043000CFE5D4E0DEBFCDBF64EF71E080E090E0B7
:100440000E94CF00A89588E190E02FE00FB6F894C5
:10045000A89581BD0FBE21BD929A8A9885B782600A
:1004600085BF8BB780648BBF939A8B9885B7886064
:1004700085BF8BB780688BBF15BC85B5822B85BDCA
:1004800089B7806889BF87E283BD0E94C40088E382
:1004900090E00E9431108C01C801AA2797FDA09519
:1004A000BA2FBC01CD010E946F1317FF06C020E0D8
:1004B00030E040E857E40E9431122FE632E143E891
:1004C0005AE30E940714DC01CB018093040190934E
:1004D0000501A0930601B09307018AE390E00E9412
:1004E00031108C01C801AA2797FDA095BA2FBC0135
:1004F000CD010E946F1317FF06C020E030E040E8F6
:1005000057E40E9431122FE632E143E85AE30E9499
:100510000714DC01CB018093080190930901A0939B
:100520000A01B0930B018CE390E00E9431108C0122
:10053000C801AA2797FDA095BA2FBC01CD010E9442
:100540006F1317FF06C020E030E040E857E40E9438
:1005500031122FE632E143E85AE30E940714DC012E
:10056000CB0180930C0190930D01A0930E01B093E9
:100570000F018EE390E00E9431108C01C801AA2780
:1005800097FDA095BA2FBC01CD010E946F1317FFF4
:1005900006C020E030E040E857E40E94311260934A
:1005A000100170931101809312019093130180E464
:1005B00090E00E9431108C01C801AA2797FDA095F8
:1005C000BA2FBC01CD010E946F1317FF06C020E0B7
:1005D00030E040E857E40E943112609314017093B8
:1005E0001501809316019093170182E490E00E9418
:1005F00031108C01C801AA2797FDA095BA2FBC0124
:10060000CD010E946F1317FF06C020E030E040E8E4
:1006100057E40E9431122FE632E143E85AE30E9488
:100620000714DC01CB018093180190931901A0936A
:100630001A01B0931B011092E4001092E500109291
:10064000E6001092E7001092E8001092E900109284
:10065000EA001092EB001092EC001092ED00109264
:10066000EE001092EF001092F0001092F100109244
:10067000F2001092F30080E090E0A0E0B0E0809300
:10068000F4009093F500A093F600B093F7008093E8
:10069000000190930101A0930201B09303018093A4
:1006A000F8009093F900A093FA00B093FB008093B8
:1006B000FC009093FD00A093FE00B093FF000E9409
:1006C000B90E60E081E00E94C60381B3806681BB01
:1006D000959A969884B38F7384BB85B3806C85BBE1
:1006E0001ABA8EEF8BBB789481E080933F0180E64D
:1006F00090E00E946E0F82E390E00E943110909390
:100700001E0180931D0184E390E00E9431109093BC
:10071000B9008093B80086E390E00E943110909376
:10072000E2008093E1001092DC00F89484E690E00F
:100730000E94291078948F3F71F00E94700881E226
:1007400092E6A0E7B0E080931F0190932001A09370
:100750002101B093220164EF71E080E090E00E94FB
:10076000CF00A8958FE191E00E94C2086FE18FE170
:1007700091E00E94880FF5CF97B1907F97B9982F9D
:100780009F7087B1892B87B9369A08953E9A96B1A2
:100790009F6C96B9982F90958AB389238ABB8BB3A7
:1007A00089238BBB80E00E94BC0308951F920F92A7
:1007B0000FB60F9211248F939F9384B195B19093AC
:1007C000CB008093CA00369A9F918F910F900FBEF5
:1007D0000F901F90189508952F923F924F925F921D
:1007E0006F927F928F929F92AF92BF92CF92DF9241
:1007F000EF92FF920F931F93CF93DF93EC01E8806A
:10080000F9800A811B818C819D81AE81BF819C0111
:10081000AD01C801B7010E9430125B016C018C89E7
:100820009D89AE89BF892AE037ED43E25BE3BC01D5
:10083000CD010E9407147B018C016C847D848E8421
:100840009F84A4019301C601B5010E943112DC010D
:10085000CB019C01AD01C801B7010E940714DC0166
:10086000CB0120E030E040E05FE3BC01CD010E941D
:1008700007147B018C0188859985AA85BB859C011D
:10088000AD01C801B7010E9431121B012C01A40166
:100890009301C601B5010E943012DC01CB0120E0BA
:1008A00030E048EC53E4BC01CD010E9407143B0149
:1008B0004C01AC86BD86CE86DF86888D998DAA8D4B
:1008C000BB8DA6019501BC01CD010E9407147B01DF
:1008D0008C018C8D9D8DAE8DBF8DA4019301BC01CB
:1008E000CD010E940714DC01CB019C01AD01C801C0
:1008F000B7010E943112DC01CB01A2019101BC01C0
:10090000CD010E9431125B016C01688B798B8A8B5F
:100910009B8BECA0FDA00EA11FA1A80197010E9436
:100920009613682E181664F088A199A1AAA1BBA1FC
:100930009C01AD01C601B5010E9493138823BCF44C
:10094000161464F0E8A0F9A00AA11BA1A801970160
:10095000C601B5010E94931388236CF4E88AF98AD2
:100960000A8B1B8BE886F9860A871B8704C02886BA
:1009700039864A865B86DF91CF911F910F91FF9058
:10098000EF90DF90CF90BF90AF909F908F907F902F
:100990006F905F904F903F902F900895AF92BF92CD
:1009A000CF92DF92EF92FF920F931F935B016C0146
:1009B00079018A010E949613181664F017FB1095AE
:1009C00017F91095A8019701C601B5010E9493136C
:1009D00088231CF4A801970102C0A6019501CA0151
:1009E000B9011F910F91FF90EF90DF90CF90BF90D2
:1009F000AF900895AF92BF92CF92DF92EF92FF92A5
:100A00000F931F93CF93DF93EC01E880F9800A8165
:100A10001B818C819D81AE81BF819C01AD01C8018C
:100A2000B7010E943012DC01CB01E888F9880A89FD
:100A30001B899C01AD01C801B7010E9407145B012D
:100A40006C01688779878A879B87EC8CFD8C0E8D7B
:100A50001F8DA80197010E949613181664F017FBCA
:100A6000109517F91095A8019701C601B5010E94CC
:100A7000931388231CF4A801970102C0A6019501D5
:100A8000288739874A875B872C873D874E875F8712
:100A9000DF91CF911F910F91FF90EF90DF90CF905A
:100AA000BF90AF9008958F929F92AF92BF92CF92D6
:100AB000DF92EF92FF920F931F93CF93DF93CDB707
:100AC000DEB74C015A016B018F859889A989BA89D3
:100AD00023ED3DE442E95FE3BC01CD010E94071430
:100AE0007B018C018B899C89AD89BE892CEB34E715
:100AF00043ED5EE3BC01CD010E940714DC01CB0194
:100B00009C01AD01C801B7010E9430127B018C012C
:100B10002AE333E24AE85DE3C601B5010E94071407
:100B2000DC01CB019C01AD01C801B7010E9431126B
:100B30007B018C018F89988DA98DBA8D29ED35E2C5
:100B40004AE05EE3BC01CD010E940714DC01CB0149
:100B50009C01AD01C801B7010E9431127B018C01DB
:100B60008B8D9C8DAD8DBE8D2AE333E24AE85DE32B
:100B7000BC01CD010E940714DC01CB019C01AD0139
:100B8000C801B7010E9431129B01AC018F85988981
:100B9000A989BA898B8B9C8BAD8BBE8B2F87388BA9
:100BA000498B5A8B8F89988DA98DBA8D8B8F9C8F8D
:100BB000AD8FBE8FAF8AB88EC98EDA8E80E1D40138
:100BC000EFE0F0E0EC0FFD1F01900D928A95E1F748
:100BD000C401DF91CF911F910F91FF90EF90DF90B3
:100BE000CF90BF90AF909F908F900895AF92BF929B
:100BF000CF92DF92EF92FF920F931F93CF93DF93E9
:100C0000EC0188819981AA81BB812C813D814E8133
:100C10005F81821B930BA40BB50BBC01CD010E941D
:100C20006F135B016C0160937E0070937F00809373
:100C30008000909381008C819D81AE81BF81288549
:100C400039854A855B85821B930BA40BB50BBC01D0
:100C5000CD010E946F13DC01CB018C8B9D8BAE8B81
:100C6000BF8B88859985AA85BB852C853D854E855A
:100C70005F85821B930BA40BB50BBC01CD010E94B9
:100C80006F13DC01CB01EC88FD880E891F899C0164
:100C9000AD01C801B7010E943012DC01CB01809385
:100CA000820090938300A0938400B093850088A174
:100CB00099A1AAA1BBA19C01AD01C601B5010E94E9
:100CC00007145B016C01E8A8F9A80AA91BA9A801EF
:100CD00097010E949613181664F017FB109517F9E8
:100CE0001095A8019701C601B5010E9493138823AE
:100CF0001CF4A801970102C0A6019501209386006B
:100D00003093870040938800509389008091DD00E4
:100D1000882309F0C1C08091DC00813069F48091A2
:100D2000500290915102AA2797FDA095BA2FBC01BD
:100D3000CD010E946F132EC08091DC00823009F03B
:100D4000CBC088A999A9AAA9BBA920E030EC4FE79C
:100D500054E4BC01CD010E947B126B017C01009127
:100D6000CA001091CB00C801AA2797FDA095BA2F01
:100D7000BC01CD010E946F1317FF06C020E030E0D8
:100D800040E857E40E9431129B01AC01C701B60153
:100D90000E9407149B01AC0160938600709387004A
:100DA00080938800909389008091E300882359F014
:100DB000DA01C901B0588093860090938700A09310
:100DC0008800B0938900E0908600F0908700009141
:100DD000880010918900888D998DAA8DBB8D9C010A
:100DE000AD01C801B7010E9430125B016C01ECA893
:100DF000FDA80EA91FA9A80197010E949613181615
:100E000064F017FB109517F91095A8019701C6011A
:100E1000B5010E94931388231CF4A801970102C016
:100E2000A6019501888D998DAA8DBB8DBC01CD0140
:100E30000E9431125B016C01609386007093870001
:100E40008093880090938900E8A8F9A80AA91BA9B3
:100E5000A80197010E949613181664F017FB1095CD
:100E600017F91095A8019701C601B5010E949313C7
:100E700088231CF4A801970102C0A60195012093C4
:100E80008600309387004093880050938900288F14
:100E9000398F4A8F5B8F20C080E090E0A0E0B0E007
:100EA0008093860090938700A0938800B093890078
:100EB0008C8B9D8BAE8BBF8B888F998FAA8FBB8FAE
:100EC0008093820090938300A0938400B093850068
:100ED000888B998BAA8BBB8BE0908600F090870063
:100EE00000918800109189008C899D89AE89BF8905
:100EF0009C01AD01C801B7010E9430127B018C0139
:100F00008CA19DA1AEA1BFA19C01AD01C801B701FB
:100F10000E9407147B018C01609386007093870008
:100F20008093880090938900809182009091830043
:100F3000A0918400B09185009C01AD01C801B7016A
:100F40000E9430127B018C0188A599A5AAA5BBA59A
:100F50009C01AD01C801B7010E940714DC01CB015F
:100F60008093860090938700A0938800B0938900B7
:100F70002AE037ED43E25BE3BC01CD010E94071498
:100F8000DC01CB01E888F9880A891B899C01AD0145
:100F9000C801B7010E943112DC01CB018C8F9D8FFB
:100FA000AE8FBF8FAC8CBD8CCE8CDF8CECA4FDA43F
:100FB0000EA51FA5A8019701C601B5010E949613B1
:100FC000181664F017FB109517F91095A8019701F2
:100FD000C601B5010E94931388231CF4A801970150
:100FE00002C0A60195012C8F3D8F4E8F5F8F8C8D97
:100FF0009D8DAE8DBF8D888B998BAA8BBB8B888581
:101000009985AA85BB858C879D87AE87BF878C8194
:101010009D81AE81BF8188879987AA87BB87DF9131
:10102000CF911F910F91FF90EF90DF90CF90BF90E5
:10103000AF900895CF93C0E080914601882389F056
:10104000EC2FFF27EA5BFE4F80810E94C90ECF5F25
:10105000EC2FFF27EA5BFE4F8081882311F0CF3F02
:1010600079F7CF91089588E10FB681BD11BC0FBE0D
:10107000F894A6E4B1E0FD0101900020E9F7EA1B35
:10108000FB0BAF0164E670E0CD010E94491078943B
:10109000A89588E190E02FE00FB6F894A89581BD5F
:1010A0000FBE21BD08956AE08FE191E00E94880F94
:1010B00067E670E08FE191E00E94DF10892B69F014
:1010C0006FE171E086E491E00E94D4106BE670E07D
:1010D00086E491E00E94D410E6CF0E943308089580
:1010E0000F931F93CF93C0E088E10FB681BD11BC71
:1010F0000FBEF894CF3F79F00C2F1127C8018C59FF
:101100009F4F0E9429100A5B1E4FF801808388239D
:1011100011F0CF5FEFCF7894A89588E190E02FE0B1
:101120000FB6F894A89581BD0FBE21BDCF911F9138
:101130000F9108950F931F93CF9388E10FB681BD50
:1011400011BC0FBEF894C0E00C2F11276FEFC8013F
:101150008C599F4F0E943E100A5B1E4FF80110826F
:10116000CF5FCF3F89F77894A89588E190E02FE092
:101170000FB6F894A89581BD0FBE21BDCF911F91E8
:101180000F9108950F931F93CF93DF93EC01888104
:10119000813209F016C4898199278236910509F4B4
:1011A00010C183369105ACF48435910509F4FBC375
:1011B000853591052CF48035910509F412C201C4DE
:1011C0008635910509F485C18A35910509F4DAC39C
:1011D000F8C38237910509F419C18337910544F4A6
:1011E0008A36910509F414C18D36910551F0E9C391
:1011F0008737910509F4D8C18A37910509F46BC383
:10120000E0C38A8199278A369105B9F08B3691051A
:1012100024F48136910569F0D4C38037910531F00B
:101220008337910509F0CDC381E004C01092DC0042
:10123000C8C382E08093DC00C4C381E08093DC00FB
:10124000BAC0809150029091510290931E018093F8
:101250001D01F89460911D0170911E0182E390E0E0
:101260000E945E10789498C0809150029091510233
:101270009093B9008093B800F8946091B800709191
:10128000B90084E390E00E945E10789485C080915C
:101290005002909151029093E2008093E100F89403
:1012A0006091E1007091E20086E390E00E945E10A0
:1012B000789472C0CF9953C0CE9951C089B3992701
:1012C00025E0969587952A95E1F79C01217030706D
:1012D00080FD45C03093510220935002309351025B
:1012E0002093500225C06AEF70E080E090E00E94F9
:1012F000CF0082B390E4892782BB80915002909105
:101300005102892B31F460ED77E080E090E00E949B
:10131000CF00CF9996CFCE99A7CFCD99B8CF809156
:101320005002909151020196909351028093500285
:101330008091140190911501A0911601B0911701AF
:10134000BC01CD010E945213DC01CB019C018091B4
:10135000500290915102281739072CF61DC0CF99E1
:1013600005C080911D0190911E0106C0CE990AC052
:101370008091B8009091B9009093510280935002EF
:1013800081E008C0CD9905C08091E1009091E20014
:10139000F3CF82E08093DC0080918A0090918B00F3
:1013A000019690938B0080938A00892B21F482B35D
:1013B00090E4892782BB0E944C0F882309F47ACFDE
:1013C00000C38A81992780379105A1F08137910563
:1013D0003CF485369105A1F08C36910571F0F1C28F
:1013E0008237910521F08437910569F0EAC20E94A5
:1013F0005308E7C20E945B0EE4C20E947008E1C27B
:101400000E949A08DEC20E941A08DBC2F894FFCF3D
:101410008A8199278937910531F18A37910524F41A
:101420008837910529F0CDC28A379105B9F1C9C233
:10143000CE0103960E94FC0F9093510280935002BC
:10144000809150029091510290931E0180931D0152
:10145000F89460911D0170911E0182E390E00E945A
:101460005E107894AEC2CE0103960E94FC0F90935A
:1014700051028093500280915002909151029093BA
:10148000B9008093B800F8946091B8007091B900E9
:1014900084E390E00E945E10789493C2CE0103969C
:1014A0000E94FC0F90935102809350028091500251
:1014B000909151029093E2008093E100F894609142
:1014C000E1007091E20086E390E00E945E10789463
:1014D00078C28091DC00813049F4CE0102960E94EE
:1014E000FC0F90935102809350026BC28091DC00FC
:1014F000882309F066C24AE050E060E070E0CE0167
:1015000002960E940011DC01CB018093E4009093CD
:10151000E500A093E600B093E70082B390E489274A
:1015200082BB2091E8003091E9004091EA0050919F
:10153000EB008091E4009091E500A091E600B0916D
:10154000E700281739074A075B0709F43AC262E344
:1015500070E080E090E00E94CF002AE030E04AEBAB
:1015600050E06091E8007091E9008091EA0090916C
:10157000EB000E9495100E946E0F80E20E94C90E3F
:101580002AE030E04AEB50E06091E4007091E50021
:101590008091E6009091E7000E9495100E946E0FE6
:1015A0008DE00E94C90EB9CF8A81992782339105B7
:1015B00079F0833391051CF4C19739F002C283336B
:1015C000910549F0C49751F0FCC1C999FECFF9C10A
:1015D000CA99FECFF6C1CB99FECFF3C1CC99FECF0D
:1015E000F0C18A8199278735910509F408C18835AA
:1015F00091054CF48534910509F42DC1853591058B
:1016000009F4D1C0DEC18437910569F085379105B1
:101610002CF48536910509F486C0D3C1873791052E
:1016200009F441C0CEC1CE0103960E94FC0FAA2747
:1016300097FDA095BA2FBC01CD010E946F13DC016C
:10164000CB012FE632E143E85AE3BC01CD010E9411
:101650000714DC01CB018093040190930501A09352
:101660000601B0930701F89480910401909105015F
:10167000A0910601B091070120E030E04AE754E470
:10168000BC01CD010E940714DC01CB01BC01CD01DE
:101690000E945213DC01CB01BC0188E390E00E9460
:1016A0005E1078948EC1CE0103960E94FC0FAA278B
:1016B00097FDA095BA2FBC01CD010E946F13DC01EC
:1016C000CB012FE632E143E85AE3BC01CD010E9491
:1016D0000714DC01CB018093080190930901A093CA
:1016E0000A01B0930B01F8948091080190910901CF
:1016F000A0910A01B0910B0120E030E04AE754E4E8
:10170000BC01CD010E940714DC01CB01BC01CD015D
:101710000E945213DC01CB01BC018AE390E00E94DD
:101720005E1078944EC1CE0103960E94FC0FAA274A
:1017300097FDA095BA2FBC01CD010E946F13DC016B
:10174000CB012FE632E143E85AE3BC01CD010E9410
:101750000714DC01CB0180930C0190930D01A09341
:101760000E01B0930F01F89480910C0190910D013E
:10177000A0910E01B0910F0120E030E04AE754E45F
:10178000BC01CD010E940714DC01CB01BC01CD01DD
:101790000E945213DC01CB01BC018CE390E00E945B
:1017A0005E1078940EC1CE0103960E94FC0FAA270A
:1017B00097FDA095BA2FBC01CD010E946F13DC01EB
:1017C000CB018093100190931101A0931201B0936B
:1017D0001301F8948091100190911101A0911201D0
:1017E000B0911301BC01CD010E945213DC01CB0169
:1017F000BC018EE390E00E945E107894E2C0CE01BE
:1018000003960E94FC0FAA2797FDA095BA2FBC0152
:10181000CD010E946F13DC01CB01809314019093E2
:101820001501A0931601B0931701F894809114014B
:1018300090911501A0911601B0911701BC01CD0145
:101840000E945213DC01CB01BC0180E490E00E94B5
:101850005E107894B6C0CE0103960E94FC0FAA27B2
:1018600097FDA095BA2FBC01CD010E946F13DC013A
:10187000CB012FE632E143E85AE3BC01CD010E94DF
:101880000714DC01CB018093180190931901A093F8
:101890001A01B0931B01F8948091180190911901DD
:1018A000A0911A01B0911B0120E030E04AE754E416
:1018B000BC01CD010E940714DC01CB01BC01CD01AC
:1018C0000E945213DC01CB01BC0182E490E00E9433
:1018D0005E10789476C0F894109242011092430101
:1018E00010924401109245011092E4001092E5001C
:1018F0001092E6001092E7001092E4001092E500CA
:101900001092E6001092E7001092E8001092E900B1
:101910001092EA001092EB001092EC001092ED0091
:101920001092EE001092EF001092F0001092F10071
:101930001092F2001092F30080E090E0A0E0B0E09E
:101940008093F4009093F500A093F600B093F70015
:101950008093000190930101A0930201B0930301D1
:101960008093F8009093F900A093FA00B093FB00E5
:101970008093FC009093FD00A093FE00B093FF00C5
:1019800078941FC06DE670E0CE0102960E94DF10D1
:10199000892BB9F4F89460E070E08EEF91E00E943A
:1019A0005E1078940EC08A8199278033910519F0D2
:1019B000C19721F006C010923F0103C081E08093DF
:1019C0003F0188818F3309F06CC189819927863561
:1019D000910509F441C0873591054CF4893491058E
:1019E00009F407C18035910509F465C057C18A36ED
:1019F000910509F4CFC08637910509F04FC18A815E
:101A000099278037910521F08337910571F046C100
:101A10002AE030E04AEB50E06091E8007091E90084
:101A20008091EA009091EB0014C08091F8009091B1
:101A3000F900A091FA00B091FB00BC01CD010E9419
:101A40005213DC01CB012AE030E04AEB50E0BC014C
:101A5000CD010E949510CAC08A81992780379105CF
:101A600021F08337910571F019C12AE030E04AEB8B
:101A700050E06091E4007091E5008091E600909163
:101A8000E700E7CF8091E300882361F08091500266
:101A9000909151024AE050E06AEB70E09095819598
:101AA0009F4FA2C04AE050E06AEB70E08091500284
:101AB0009091510299C08A8199278735910509F43F
:101AC0004FC08835910544F48534910509F455C01B
:101AD00085359105C1F1E2C08437910559F085370C
:101AE000910524F48536910509F1D8C08737910511
:101AF00071F0D4C00FE111E023E047E060910401F0
:101B00007091050180910601909107010CC00FE1D1
:101B100011E023E047E06091080170910901809194
:101B20000A0190910B010E94C11260C00FE111E007
:101B300023E047E060910C0170910D0180910E014E
:101B400090910F01F0CF0FE111E023E047E06091A9
:101B50001001709111018091120190911301E3CF56
:101B60000FE111E023E047E060911401709115014D
:101B70008091160190911701D6CF0FE111E023E07B
:101B800047E0609118017091190180911A019091BC
:101B90001B01C9CF8A81992789379105A1F08A371E
:101BA000910524F48837910529F078C08A3791058A
:101BB00099F074C04AE050E06FE171E080911D013E
:101BC00090911E0111C04AE050E06FE171E08091F8
:101BD000B8009091B90008C04AE050E06FE171E0B0
:101BE0008091E1009091E2000E9470100E946E0FBF
:101BF00055C08BE10E94C90E8BE50E94C90E82E39D
:101C00000E94C90E8AE40E94C90E8FE291E00E94F0
:101C1000CB0F80E291E00E94CB0F8CE291E00E941A
:101C2000CB0F87E191E00E94CB0F8DE00E94C90E9F
:101C300084E091E00E94CB0F8FE091E00E94CB0FF7
:101C4000F8948EEF91E00E943110909341018093BF
:101C5000400178944AE050E06FE171E080914001EA
:101C6000909141010E9470108FE191E00E946E0FEF
:101C70008DE00E94C90E8DE00E94C90E89EE90E0B1
:101C80000E94CB0F82ED90E00E94CB0F8DEB90E095
:101C90000E94CB0F87EA90E00E94CB0F8DE00E945C
:101CA000C90E85E790E00E946E0F9698DF91CF9164
:101CB0001F910F910895EF92FF920F931F93CF936F
:101CC00010E0012FC12F36E4E32E31E0F32EF701AF
:101CD00001900020E9F73197EE15FF0509F443C0A4
:101CE000EC2FFF27EA5BFE4F80818D3059F520E015
:101CF0001C1778F4A12FBB27AA5BBE4F9C2F911B0A
:101D0000E22FFF27EA5BFD4F8D9180832F5F91507B
:101D1000B9F7E22FFF27EA5BFD4F10821C2F1F5FF0
:101D20000E944C0F8823F9F468E770E086E492E0A3
:101D30000E94DF10892B11F401E004C086E492E0D8
:101D40000E94C208CF5F8C2F9927F70101900020D5
:101D5000E9F73197E654F1408E179F0708F4C0CF9A
:101D6000002309F0ADCFCF911F910F91FF90EF901D
:101D7000089580E189B988E98AB986E880BD80E064
:101D80008093AD008093AC008093B7008093B60041
:101D90000895282F9091B6009F5F97708091B700AB
:101DA0009817E1F3E92FFF27E255FF4F2083909327
:101DB000B600559A08951F920F920FB60F921124F4
:101DC0002F933F934F935F936F937F938F939F9343
:101DD000AF93BF93EF93FF939CB1E091AC00EF5FA3
:101DE000EF71E093AC008091AD00E81721F0FF2780
:101DF000E457FF4F908380913F01882319F0892F8A
:101E00000E94C90EFF91EF91BF91AF919F918F9169
:101E10007F916F915F914F913F912F910F900FBEE6
:101E20000F901F9018951F920F920FB60F921124CA
:101E30008F939F93EF93FF939091B6008091B7009B
:101E4000981769F08091B7008F5F87708093B70013
:101E5000E82FFF27E255FF4F80818CB901C05598CC
:101E6000FF91EF919F918F910F900FBE0F901F9058
:101E700018959091AC008091AD009817D1F38091A6
:101E8000AD008F5F8F718093AD00E82FFF27E4577F
:101E9000FF4F80819927089520E030E09091AC00B9
:101EA0008091AD00981711F021E030E0C90108954C
:101EB00020E030E09091B6008091B700981711F0C3
:101EC00021E030E0C901089580E00E94C90E8DE054
:101ED0000E94C90E8AE00E94C90E08951F93CF93F5
:101EE000DF93EC0110E08881882361F0FE01E10FAF
:101EF000F11D80810E94C90E1F5FFE01E10FF11DDF
:101F00008081F2CF812F9927DF91CF911F91089582
:101F1000CF92DF92FF920F931F93CF93DF93CDB7B2
:101F2000DEB721970FB6F894DEBF0FBECDBF8C0190
:101F3000F62E90E09617C8F4680199830E94390F35
:101F4000F601808399818D3021F08A3011F0882349
:101F500031F4F60110829F5F892F99270EC09F5F91
:101F60000894C11CD11C9F1540F3892F9927080F95
:101F7000191F01501040F801108221960FB6F894F5
:101F8000DEBF0FBECDBFDF91CF911F910F91FF90AC
:101F9000DF90CF900895BC018FE191E00E94E9109D
:101FA0008FE191E00E946E0F08950F931F93182FF9
:101FB000062F8BE10E94C90E8BE50E94C90E4AE0F4
:101FC00050E06FE171E0812F99270E9470100E940C
:101FD0006E0F8BE30E94C90E4AE050E06FE171E0A2
:101FE000802F99270E9470100E946E0F88E40E9433
:101FF000C90E1F910F910895FC0188279927E89435
:1020000021912223F1F02032D9F32930C9F32A306B
:10201000B9F32C30A9F32D3099F3263789F32B32FD
:1020200019F02D3221F468942191222351F02033AC
:1020300044F02A3334F420530E94CC10820F911DB7
:10204000F3CF8115910521F01EF4809590950196AE
:102050000895E199FECF9FBB8EBBE09A99278DB37F
:102060000895E199FECF9FBB8EBBE09A01960DB219
:102070009FBB8EBBE09A802D9DB30895E199FECF62
:102080009FBB8EBB6DBB0FB6F894E29AE19A0FBE70
:1020900008954115510589F0DC018FB7E199FECF14
:1020A0007FBB6EBB0D900DBAF894E29AE19A8FBF98
:1020B0006F5F7F4F4150504089F70895FFEF0FB693
:1020C000E199FECF9FBB8EBB6DBBF894E29AE19A7B
:1020D0000FBEF0FF08958F5F9F4F672FFF27F0CF50
:1020E000E62FF72F2E2F3F2FE8944230CCF04532C9
:1020F000BCF44A3029F497FB1EF4909581959F4FCC
:10210000642F77270E94AA15805D8A330CF0895DC1
:102110008193862F972F009799F716F45DE25193DC
:10212000932F822F10820C94F010F52FE42FCF9371
:10213000FF93EF93223054F1253244F5C22FE894F7
:10214000CA3049F497FB3EF490958095709561955F
:102150007F4F8F4F9F4F2C2F332744275527FF93B7
:10216000EF930E94BE15EF91FF91605D6A330CF012
:10217000695D6193622F732F842F952F605070409B
:102180008040904041F716F4CDE2C19310828F91C8
:102190009F91CF910C94F0107AE0979F902D879F9C
:1021A000802D910D11240895FB01DC010D9000207C
:1021B000E9F7119701900D920020E1F70895FB01D6
:1021C000DC018D910190801911F40020D1F7990B59
:1021D0000895FB01DC0105900D920020E1F70895C0
:1021E000DC01FC0101900020E9F73297AE17BF0730
:1021F00030F47C916081708331976D93F7CF0895AF
:102200003F924F925F926F927F928F929F92AF9286
:10221000BF92CF92DF92EF92FF920F931F93CF93D3
:102220008C012B017A0133246115710519F0FB0132
:1022300080839183E114F10449F0C70102978397E9
:1022400028F020E030E040E050E0F7C0F801C19114
:102250008F018C2F99270E947915892BB9F7CD32E0
:1022600009F44FC0CB3209F44EC0E114F10441F13E
:10227000F0E1EF16F10421F1E114F10431F4C0337F
:1022800009F4D0C04AE0E42EF12C88E0E816F1040D
:10229000F1F1E9E0EE16F1042CF5F2E0EF16F104AD
:1022A00009F4A3C09701442737FD4095542F60E0FF
:1022B00070E080E090E80E94BE1559016A012CC0D0
:1022C000C033D1F6F8018081883711F08835A1F646
:1022D000F801C1810E5F1F4F60E1E62EF12CF2E0A4
:1022E0003F2AD3CF8AE0E816F10409F475C0E0E193
:1022F000EE16F104B9F6A12CB12CC12C28E0D22E97
:102300000BC071E0372EF801C1918F01AECFA12C27
:10231000B12CC12C90E1D92E20E030E040E050E01B
:1023200060E03701882477FC8094982C8C2F8053B0
:102330008A30A8F4C82FAC2FBB27AE15BF05CCF44C
:1023400067FD06C0A216B306C406D50658F56FEFA2
:10235000F801C1918F018C2F80538A3058F37C2F64
:1023600071547A3198F5C753AC2FBB27AE15BF0512
:102370003CF34114510441F0662309F449C0015073
:102380001040F20100831183832D992767FD4EC011
:1023900080FF31C050954095309521953F4F4F4F6C
:1023A0005F4F4BC0C401B3010E948B159B01AC0170
:1023B0002C0F311D411D511D2130F0E03F07F0E091
:1023C0004F07F0E85F0718F661E0C2CF9C2F9156E7
:1023D0009A3178F6C755AFCF3CECA32E3CECB32E28
:1023E0003CECC32E3CE0D32E97CFA12CB12CC12CBA
:1023F00080E4D82E91CF57FF20C02FEF3FEF4FEF53
:102400005FE702E210E0109353020093520215C0FE
:10241000832D992781FFBCCF02501040F201008329
:102420001183B6CF58E0E52EF12C2FCF80FFE5CFFA
:1024300020E030E040E050E8E4CFCA01B901CF919C
:102440001F910F91FF90EF90DF90CF90BF90AF90D2
:102450009F908F907F906F905F904F903F900895E6
:102460005058192EA2D101D085C1BA17620773073F
:1024700084079507B1F188F40EF410940B2EBA2F4F
:10248000A02D062E622F202D072E732F302D082E03
:10249000842F402D092E952F502DFF275523B9F05D
:1024A000591B49F0573E98F0469537952795A795C3
:1024B000F0405395C9F776F0BA0F621F731F841F5F
:1024C00030F4879577956795B795F040939517FA0F
:1024D0000F2E0895BF1BBB27BA0B620B730B840B27
:1024E000F6CFDEF67FC1592F482F372F262F9FE3D7
:1024F00080E87727662759D101D03CC1552359F090
:10250000992369F09F575F57951B33F442F4903835
:1025100011F4915805C046C191589F3F09F462C11A
:10252000BB27112462177307840730F4660F771FE7
:10253000881FBB1F915098F311D00F920FD00F92AC
:102540000DD0A0E82617370748071B0609F0A0485A
:10255000BA2F602D7F918F9100240895A0E8002468
:10256000621773078407B10528F0621B730B840B95
:10257000B1090A2A660F771F881FBB1FA69581F72E
:102580000895DF93CF931F930F93E8018C01000F01
:10259000111F1F3F31F49EE481E49993899399932D
:1025A0007AC04F9399231AF40DE209939F77022F73
:1025B00003959F938F937F936F93622F772788273D
:1025C00099270E946F139068AC019B0191E480E20F
:1025D000772766270E9455145FEF4FEF0E94F41390
:1025E0002F913F914F915F910E943112102F013036
:1025F00009F4002751E440E23327222762177307CA
:102600008407950724F00E947B121395F3CF9F93C4
:102610008F937F936F930E945213562F505D59935F
:102620000E946F132F913F914F915F910E94301242
:10263000905851E440E2332722270E9407141017D4
:1026400011F45EE259931A9511F718825F91EF9198
:10265000FF91FF93EF93452F442312F44095439548
:10266000CE01BF01861B970B142F181B90E2841715
:102670009CF455236AF021963196E40FF11D839561
:102680005A9152938A95E1F792931A95E9F704C00B
:1026900099931A95E9F718828F919F918C01CF91A8
:1026A000DF91089597FB8DD09F3738F0FEE9F91B35
:1026B000982F872F762F6B2F05C091C09695879501
:1026C00077956795F150D0F73EF490958095709589
:1026D00061957F4F8F4F9F4F0895E89403C097FBFC
:1026E0000EF4F3DFB62F672F782F892F9EE9002491
:1026F00041C097FB66D09F3760F40EF070C09FEB2F
:1027000080E8772766270895869577956795B11DA8
:1027100093959639C8F32EF4BB2319F06F5F7F4F62
:102720008F4FBB2727C00ED05EF004C00BD026F021
:1027300001C008D019F020F48FEF089580E00895CB
:1027400081E0089597FB092E052600F8689430D0A3
:10275000E89407FC07C0621773078407950721F008
:1027600008F400940794989408959A95BB0F661FF7
:10277000771F881F11249923A1F08823B2F79F3F68
:1027800059F0BB0F48F421F4002011F460FF04C09D
:102790006F5F7F4F8F4F9F4F881F9795879597F952
:1027A00008951DC09FEF80EC0895052E092607FAB5
:1027B000440F551F5F3F79F0AA27A51708F051E095
:1027C0004795880F991F9F3F31F0BB27B91708F035
:1027D00091E0879508959F919F911124E3CF6627FB
:1027E000772788279927089597FBEBDF992329F00E
:1027F0005F3F29F0552319F00AF4F1CFD3CF940F9E
:10280000151E01F4B7CF592F482F372F262FCDDFB4
:1028100001D0B0CF992339F0552329F09F575F5746
:10282000950F13F4CAF1DECF91589F3FE1F3A62F25
:1028300000241124BB2766275527F8E0A69520F42D
:10284000020E131EB41F651F220F331F441F551F96
:10285000FA95A1F7F8E0E72F7727F8E0E69520F45E
:10286000130EB41F651F7A1F330F441F551FAA1F75
:10287000FA95A1F7F82F8827F69520F4B40F651F75
:102880007A1F8E1F440F551FAA1FEE1FFF23A1F7AB
:1028900088231AF4939539F485CF000C111CBB1FC3
:1028A000661F771F881F01280895552371F199230A
:1028B00062F059F15F934F933F932F93BBD02F91C9
:1028C0003F914F915F91A3DF25C09F938F937F939B
:1028D0006F935F934F933F932F93952F842F732F75
:1028E000622FE0DEBDDD91158105710561052F9137
:1028F0003F914F915F916F917F918F919F9121F0C7
:102900009F775058E2DF50584DCF9FE380E87727FC
:1029100066270895092E99234AF052E441EB32E7E5
:10292000683173078407950758F03CCF9F7752E4CE
:102930004EEA3CEA603573078407950708F04FCFED
:102940000F925FE348EB3AEA2BE361DFFF92EF92ED
:10295000DF92CF9250E04CE096D0E4E5F0E01ED05C
:102960005F2D4E2D3D2D2C2DCF90DF90EF90FF90C1
:10297000FEE94595441F551FF51B5527406804C0C7
:102980004695379527955795FA95D2F7452F550FC8
:10299000550B2ADF0F9007FCA6CD0895092E11DFF5
:1029A000FF92EF92DF92CF92BF92AF92B02CC92EDE
:1029B000D82EE72EF62EA59018D0A590AA2071F05B
:1029C0009F938F937F936F936F2D7E2D8D2D9C2DD5
:1029D0000CD02F913F914F915F9190DDAF90BF90C0
:1029E000CF90DF90EF90FF90C5CE7ED047FB406840
:1029F00004C02F2D3E2D4D2D5C2DEF93FF930ADF4C
:102A0000FF91EF9171D0AA2707F80B24102C042610
:102A100007FA4068FF9329DDFF91992341F088234D
:102A200032F09A95BB0F661F771F881FF8CFAA94C4
:102A300001F7089597FDB6CEC4DE992309F4B2CE0E
:102A4000FF92EF92DF92CF92C92E9FE38F77E2E75A
:102A5000F0E0A4DF0C2CC92ED82EE72EF62E602D28
:102A60006E57770B872F972F3ADE5FE341E332E70C
:102A700028E1CDDE5C2D4D2D3E2D2F2DCF90DF900A
:102A8000EF90FF90EECC97FB9CDECF93DF93D52F9A
:102A9000C42F55274427332722279923D9F09F375E
:102AA000C8F0F92F67DE592F482F372F262FF63918
:102AB00068F4F8DD14DEC030CD0721F06993799316
:102AC000899399939058DF91CF91CBCC9927882700
:102AD00077276627C030CD0721F029933993499392
:102AE0005993DF91CF9146CE5591459135912591DE
:102AF0000895992369F4803269F08A3059F08C3056
:102B000049F08D3039F0893029F08B3009F408957F
:102B1000992788270895629FD001739FF001829FB3
:102B2000E00DF11D649FE00DF11D929FF00D839F5C
:102B3000F00D749FF00D659FF00D9927729FB00DF9
:102B4000E11DF91F639FB00DE11DF91FBD01CF010C
:102B500011240895AA1BBB1B51E107C0AA1FBB1F6C
:102B6000A617B70710F0A61BB70B881F991F5A9519
:102B7000A9F780959095BC01CD010895A1E21A2E88
:102B8000AA1BBB1BFD010DC0AA1FBB1FEE1FFF1F11
:102B9000A217B307E407F50720F0A21BB30BE40B61
:102BA000F50B661F771F881F991F1A9469F76095A8
:102BB0007095809590959B01AC01BD01CF01089562
:102BC00052455345540D00216273000D0076657225
:0C2BD00073696F6E002E0D002162700012
:00000001FF
